:020000040000FA
:020000000528D1
:0800080009008316FF3085009A
:1000100003018600CF30810000308B0083128601FF
:100020009701D42063309A009C009D309B009D0076
:1000300044211521EE304B211A211521EE302121CA
:1000400065216E2163009E014421031D9E0A152136
:10005000EE304B2144211521AA304B2158219F011C
:100060001A21031D9F0A1521EE3021211A21152185
:10007000AA3021212E211E08031D52281808803A7B
:1000800093001A08803A13020318482818089A00A7
:100090001808803A93001B08803A1302031C522868
:1000A00018089B001F08031D69281908803A93004F
:1000B0001C08803A130203185F2819089C001908CD
:1000C000803A93001D08803A1302031C692819081E
:1000D0009D008030C0200030F7201A0893205F3048
:1000E000C9201E08031D8D28180893200830F7200A
:1000F0001B089320C030C0200430F7201C08932038
:100100005F30C9201F08031D90281908932008306C
:10011000F7201D089320E52021280C30F7207828AF
:100120000C30F72089289500951F9D289509150802
:10013000013E95002D30C9209F282B30C92015087D
:10014000A320B92008009000900A91019201900B21
:10015000AA280800910A0A301106031DA728910158
:10016000920A0A301206031DA72809309100920056
:1001700008001208303EC9201108303EC92008008E
:100180009600F0398600F320160EF0398600F32031
:1001900008009600F03986000615F320160EF03997
:1001A00086000615F320080020308600F320E520A5
:1001B0002830C020EE200C30C020EE200130C020BE
:1001C000EE200630C020EE200800FF309300033000
:1001D0009400930BE928940BE92808001130930050
:1001E000930BF02808008615EE2086110800831274
:1001F0008900831608148312080803190800C9200F
:10020000890AF9288511831685118312080083163F
:1002100085158312080002309300930B0D29080006
:100220001D309300930B12290800F7309300930BB5
:100230001729080002211521072110210508083976
:10024000080099000830940002210B21990C031832
:10025000851510210721940B2429080008309400EB
:1002600002210721000005080839FF3E990C1021E2
:10027000940B30290800051183160511831208001C
:1002800083160515831208003B21152140211021FA
:100290000508043908009800083094003B210B2120
:1002A000980C0318051510214021940B4E290800C5
:1002B000083094003B214021000005080439FF3E2E
:1002C000980C1021940B5A2908008030C02013305C
:1002D000F720C030C0202430F72008001E08031D7E
:1002E00008001808803A93000230803A130203187D
:0E02F0000800FF309706031908008614080066
:02400E00F53F7C
:10420000453458342034003449344E34203400349A
:10421000DF3443345F3400343F3445345234523455
:104220003F345F3400342A34203454344834453425
:1042300052344D344F3420345634203432342E34FA
:10424000303420342A3400342A342034563469344B
:10425000633473347934733420343234303430344A
:0A4260003734203420342A340034AF
:00000001FF
